:107E0000F894112424B614BE2EBA8DE0822129F0F4
:107E100040E0CFD0EE27FF270994259A4EE0C9D045
:107E200020E031E082E08093C00096E09093C200B1
:107E300090E19093C40088E18093C10053E02D9AB3
:107E4000BED02D98BCD05150D1F78FD0813461F481
:107E50008CD0582F7DD083E0523821F083E0513808
:107E600009F484E77AD05CC044E1823419F045E03B
:107E7000853411F46AD054C0853541F476D0482E4B
:107E800074D0582E440C551CF2015DC0863521F487
:107E900044E05BD080E0E6CF843609F02EC074D099
:107EA00021F080E7581608F47CD0E9015ED0899370
:107EB0001197E1F7D801E9014BD0611009C0A895ED
:107EC00089915CD080BDFA9AF99A1197C1F728C0C0
:107ED00080E7581608F065D060D0F201099019903B
:107EE00041E061D0112432961297C1F7F20145E0CA
:107EF0005AD053D041E157D013C08437A1F444D0B5
:107F000027D0662039F4119750F038D0F89A80B510
:107F100024D0F9CFF201859120D01197E1F72F01FC
:107F200080E11BD092CF853741F449F411D08EE126
:107F300014D085E912D08FE095CF803299F3813546
:107F400011F448E036D004D0EBCF0FD04150E9F720
:107F50000CD0803209F02AD084E19091C00095FFC6
:107F6000FCCF8093C600A89508958091C00087FF3C
:107F7000FCCF84FFA8958091C6000895F999FECFA3
:107F8000F2BDE1BD31960895F0DF182FEEDF082F26
:107F9000D801EBDF8554682E089507B600FCFDCFAD
:107FA0000895F20143E047BFE895089548E001D005
:107FB000FFCF58E1509360004093600008958CEF2C
:107FC0008093850082EF8093840085E08093810018
:0C7FD00086B380FFFDCF86BBA895089506
:027FFE0003740A
:0400000300007E007B
:00000001FF
